:1000000012C02CC02BC02AC029C028C027C026C0BF
:1000100025C025C023C022C021C020C01FC01EC0D3
:100020001DC01CC01BC011241FBECFE5D4E0DEBF25
:10003000CDBF10E0A0E6B0E0E8E7F3E102C0059034
:100040000D92A236B107D9F710E0A2E6B0E001C0E8
:100050001D92AE38B107E1F7DDD18CC9D1CF1F9227
:100060000F920FB60F9211242F933F934F935F93EC
:100070006F937F938F939F93AF93BF93EF93FF9370
:10008000DF93CF9300D000D000D0CDB7DEB7E2E54C
:10009000F0E085E08083E0E3F0E08081882F90E06D
:1000A00021D280917B00882369F0A2E3B0E0E2E3F3
:1000B000F0E0808180618C9380917B0081508093FF
:1000C0007B0007C0A2E3B0E0E2E3F0E080818F7E36
:1000D0008C93809165008F5F8093650080916500AF
:1000E000823309F09DC010926500809162008130DA
:1000F00089F58091740090917500009751F080917E
:10010000740090917500019790937500809374002E
:100110000FC088EB80937B0084E08093620088EBC3
:100120009BE0909361008093600082E090E0F0D7C4
:1001300080917400909175002AE030E0B901E1D817
:100140008530910520F480E090E0E2D703C081E0A3
:1001500090E0DED780917200282F30E03E832D831F
:100160008D819E8183309105A1F02D813E812430C7
:100170003105C9F08D819E8182309105F1F4809125
:100180008700909188000A97909388008093870059
:1001900014C08091870090918800449790938800C4
:1001A000809387000AC080918700909188008E56C6
:1001B0009040909388008093870080916B00282F57
:1001C00030E03C832B838B819C8183309105A1F0AF
:1001D0002B813C8124303105C9F08B819C81823098
:1001E0009105F1F480918700909188000A96909390
:1001F00088008093870014C08091870090918800C8
:10020000449690938800809387000AC0809187006D
:100210009091880082599F4F909388008093870027
:1002200080918300882309F474C080918300813019
:1002300009F05AC01092830080917C008F5F8093F8
:100240007C0080916200282F30E03A8329838981E5
:100250009A818230910541F129813A81233031051B
:1002600054F489819A81009789F029813A8121305B
:10027000310599F039C089819A8183309105C1F0A7
:1002800029813A812430310511F12EC081E080931B
:10029000620084E680937B0027C082E08093620046
:1002A00081E090E035D720C081E0809362001CC0DF
:1002B000E5D710926200809187009091880090931A
:1002C00075008093740082E090E022D70DC01092F8
:1002D00062008091870090918800909375008093D0
:1002E000740082E090E014D780918300823089F41A
:1002F00080916200882369F01092620080918700EB
:1003000090918800909375008093740082E090E053
:10031000FFD6809162008330F1F4809172008130C9
:1003200059F480918700909188000A9790938800F3
:10033000809387001092720080916B00813059F495
:1003400080918700909188000A969093880080930E
:10035000870010926B0080918700909188003AEEA0
:100360008735930788F0809187009091880026EF69
:100370008831920748F486E59AEE9093880080933E
:10038000870084E680937B008091870090918800AD
:100390008A30910540F0809187009091880036EF77
:1003A0008931930748F08AE090E090938800809329
:1003B000870084E680937B008091620080936200D6
:1003C00047D280916200813041F4A2E3B0E0E2E3E1
:1003D000F0E0808180688C9307C0A2E3B0E0E2E3A4
:1003E000F0E080818F778C932696DEBFCDBFCF91D2
:1003F000DF91FF91EF91BF91AF919F918F917F918D
:100400006F915F914F913F912F910F900FBE0F9081
:100410001F901895DF93CF9300D0CDB7DEB7E7E3F9
:10042000F0E08FEF8083E8E3F0E01082E4E3F0E0B7
:100430008FE38083E5E3F0E08FE38083E1E3F0E0A6
:1004400080EF8083E2E3F0E08FE08083E3E5F0E09B
:1004500083E08083E9E5F0E081E080837894809117
:10046000870090918800909375008093740010929B
:10047000620082E090E04CD684E680937B0018D73F
:10048000809187009091880090937500809374000C
:1004900080916200282F30E03A83298389819A81F4
:1004A0008330910531F029813A812430310539F0CA
:1004B00013C0809187009091880076D6E9CF8BE0B9
:1004C000809379008CE0809378008DE080937700B2
:1004D0008AE080937600DCCF809174009091750063
:1004E00063D6D6CFDF93CF9300D000D0CDB7DEB7A1
:1004F00089838981882F90E0817090701C82009799
:1005000011F421E02C838C8180936D008981869584
:10051000882F90E0817090701B82009711F421E089
:100520002B838B818093660089818695869586953D
:10053000882F90E0817090701A82009711F421E06A
:100540002A838A8180937E0080917E00882339F1FE
:100550008091840091E08927882349F0809181006F
:100560009091820001969093820080938100809107
:1005700081009091820023E0893E920768F182E039
:10058000809383009091840081E08927882319F06B
:1005900085E080937B0081E0809384001DC01092F1
:1005A000840080918100909182000097A9F0809151
:1005B0008300823058F481E080938300109282009F
:1005C0001092810085E080937B0006C0109282002B
:1005D000109281001092830080916D0091E0892734
:1005E0008823C1F48091660091E08927882391F4E3
:1005F00080916200882331F483E08093620085E07B
:1006000080937B0081E080936C0080916C008093EC
:100610007300DBC080916200833009F0D6C0809106
:100620006600882309F44DC080916C0091E0892711
:10063000882349F08091690090916A000196909317
:100640006A00809369008091690090916A0023E1BB
:100650008938920780F080916C0091E08927882387
:1006600019F085E080937B0081E080936C0084E04A
:1006700080936B003FC08091690090916A0027E0F1
:10068000813D920758F080916B00823019F485E02B
:1006900080937B0083E080936B002CC08091690085
:1006A00090916A0021E0853F920720F180916B00D4
:1006B000882319F485E080937B0082E080936B00AF
:1006C00019C08091690090916A00009769F080914B
:1006D0006B00823038F481E080936B0085E080937A
:1006E0007B0002C010926B0010926C0010926A00A6
:1006F0001092690080916D00882309F44DC08091AB
:10070000730091E08927882349F0809170009091CF
:100710007100019690937100809370008091700039
:100720009091710023E18938920780F080917300E5
:1007300091E08927882319F085E080937B0081E090
:100740008093730084E0809372003FC080917000BA
:100750009091710027E0813D920758F080917200DE
:10076000823019F485E080937B0083E080937200EF
:100770002CC0809170009091710021E0853F92071C
:1007800020F180917200882319F485E080937B002A
:1007900082E08093720019C0809170009091710086
:1007A000009769F080917200823038F481E0809384
:1007B000720085E080937B0002C01092720010925C
:1007C000730010927100109270000F900F900F90B4
:1007D0000F90CF91DF910895DF93CF93CDB7DEB720
:1007E00027970FB6F894DEBF0FBECDBF9E838D83D3
:1007F0008CE890E09A83898313C01C821B8209C015
:100800008D819E810097D9F08B819C8101969C837C
:100810008B832B813C8189819A812817390780F34A
:100820001F828D819E81009711F081E08F838D81E1
:100830009E8101979E838D838F818823F1F6279671
:100840000FB6F894DEBF0FBECDBFCF91DF910895F4
:10085000DF93CF93CDB7DEB727970FB6F894DEBFFF
:100860000FBECDBF898380917A008F5F80937A001D
:1008700080917D008F5F80937D0080917D00893C19
:1008800050F09091890081E08927882F90E0809333
:10089000890010927D0080917A00843010F01092CF
:1008A0007A00A8E3B0E0E8E3F0E0808181608C9317
:1008B000A8E3B0E0E8E3F0E0808184608C93A8E3F3
:1008C000B0E0E8E3F0E0808182608C93A8E3B0E0E0
:1008D000E8E3F0E0808188608C938981843049F579
:1008E0008091890091E08927882301F184E0809339
:1008F0007A0081E090E00CD48091600090916100DA
:10090000009751F080916000909161000197909361
:100910006100809360000DC088EB9BE090936100C4
:100920008093600088EE80937B0003C082E090E0BB
:10093000EFD380917A00882F90E0FC01EA58FF4FB6
:100940008081282F30E03F832E838E819F818630E7
:10095000910509F480C12E813F812730310524F5AE
:100960008E819F818230910509F4ADC02E813F8137
:100970002330310564F48E819F81009709F43FC0D4
:100980002E813F812130310509F46BC0F3C28E8185
:100990009F818430910509F4FAC02E813F81253072
:1009A00031050CF026C1C1C08E819F818A3091052E
:1009B00009F419C22E813F812B3031056CF48E81F0
:1009C0009F818830910509F4AAC12E813F81293089
:1009D00031050CF0D6C171C18E819F818C3091059B
:1009E00009F465C22E813F812C3031050CF42DC2F3
:1009F0008E819F818D30910509F48BC2BBC2A5E326
:100A0000B0E0E5E3F0E080818F7D8C93A8E3B0E077
:100A1000E8E3F0E080818F7E8C93A5E3B0E0E5E32E
:100A2000F0E080818E7F8C93A5E3B0E0E5E3F0E019
:100A300080818B7F8C93A5E3B0E0E5E3F0E08081DB
:100A4000877F8C93A5E3B0E0E5E3F0E080818F7EC3
:100A50008C93A8E3B0E0E8E3F0E0808180628C93BF
:100A600089C2A5E3B0E0E5E3F0E0808180628C9389
:100A7000A8E3B0E0E8E3F0E080818F7E8C93A5E30B
:100A8000B0E0E5E3F0E080818E7F8C93A5E3B0E0F9
:100A9000E5E3F0E0808184608C93A5E3B0E0E5E3DA
:100AA000F0E0808188608C93A5E3B0E0E5E3F0E0BE
:100AB000808180618C93A8E3B0E0E8E3F0E080817E
:100AC00080628C9357C2A5E3B0E0E5E3F0E080815B
:100AD0008F7D8C93A8E3B0E0E8E3F0E080818F7E27
:100AE0008C93A5E3B0E0E5E3F0E0808181608C9336
:100AF000A5E3B0E0E5E3F0E080818B7F8C93A5E394
:100B0000B0E0E5E3F0E08081877F8C93A5E3B0E07F
:100B1000E5E3F0E0808180618C93A8E3B0E0E8E356
:100B2000F0E080818F7D8C9325C2A5E3B0E0E5E302
:100B3000F0E080818F7D8C93A8E3B0E0E8E3F0E003
:100B400080818F7E8C93A5E3B0E0E5E3F0E08081C7
:100B50008E7F8C93A5E3B0E0E5E3F0E080818B7FAE
:100B60008C93A5E3B0E0E5E3F0E0808188608C93AE
:100B7000A5E3B0E0E5E3F0E0808180618C93A8E339
:100B8000B0E0E8E3F0E080818F7D8C93F3C1A5E3D2
:100B9000B0E0E5E3F0E0808180628C93A8E3B0E010
:100BA000E8E3F0E080818F7E8C93A5E3B0E0E5E39D
:100BB000F0E080818E7F8C93A5E3B0E0E5E3F0E088
:100BC000808184608C93A5E3B0E0E5E3F0E0808170
:100BD00088608C93A5E3B0E0E5E3F0E080818F7E50
:100BE0008C93A8E3B0E0E8E3F0E080818F7D8C9304
:100BF000C1C1A5E3B0E0E5E3F0E080818F7D8C9397
:100C0000A8E3B0E0E8E3F0E0808180618C93A5E3A5
:100C1000B0E0E5E3F0E080818E7F8C93A5E3B0E067
:100C2000E5E3F0E080818B7F8C93A5E3B0E0E5E322
:100C3000F0E0808188608C93A5E3B0E0E5E3F0E02C
:100C400080818F7E8C93A8E3B0E0E8E3F0E08081C0
:100C50008F7D8C938FC1A5E3B0E0E5E3F0E0808168
:100C60008F7D8C93A8E3B0E0E8E3F0E080818061C1
:100C70008C93A5E3B0E0E5E3F0E080818E7F8C9378
:100C8000A5E3B0E0E5E3F0E080818B7F8C93A5E302
:100C9000B0E0E5E3F0E08081877F8C93A5E3B0E0EE
:100CA000E5E3F0E080818F7E8C93A8E3B0E0E8E399
:100CB000F0E080818F7D8C935DC1A5E3B0E0E5E33A
:100CC000F0E080818F7D8C93A8E3B0E0E8E3F0E072
:100CD00080818F7E8C93A5E3B0E0E5E3F0E0808136
:100CE0008E7F8C93A5E3B0E0E5E3F0E08081846043
:100CF0008C93A5E3B0E0E5E3F0E0808188608C931D
:100D0000A5E3B0E0E5E3F0E0808180618C93A8E3A7
:100D1000B0E0E8E3F0E0808180628C932BC1A5E332
:100D2000B0E0E5E3F0E080818F7D8C93A8E3B0E054
:100D3000E8E3F0E080818F7E8C93A5E3B0E0E5E30B
:100D4000F0E080818E7F8C93A5E3B0E0E5E3F0E0F6
:100D500080818B7F8C93A5E3B0E0E5E3F0E08081B8
:100D6000877F8C93A5E3B0E0E5E3F0E080818F7EA0
:100D70008C93A8E3B0E0E8E3F0E080818F7D8C9372
:100D8000F9C0A5E3B0E0E5E3F0E080818F7D8C93CE
:100D9000A8E3B0E0E8E3F0E080818F7E8C93A5E3E8
:100DA000B0E0E5E3F0E080818E7F8C93A5E3B0E0D6
:100DB000E5E3F0E080818B7F8C93A5E3B0E0E5E391
:100DC000F0E0808188608C93A5E3B0E0E5E3F0E09B
:100DD00080818F7E8C93A8E3B0E0E8E3F0E080812F
:100DE0008F7D8C93C7C0A5E3B0E0E5E3F0E08081A0
:100DF00080628C93A8E3B0E0E8E3F0E0808180615A
:100E00008C93A5E3B0E0E5E3F0E0808181608C9312
:100E1000A5E3B0E0E5E3F0E0808184608C93A5E396
:100E2000B0E0E5E3F0E0808188608C93A5E3B0E07A
:100E3000E5E3F0E0808180618C93A8E3B0E0E8E333
:100E4000F0E0808180628C9395C0A5E3B0E0E5E39B
:100E5000F0E080818F7D8C93A8E3B0E0E8E3F0E0E0
:100E6000808180618C93A5E3B0E0E5E3F0E08081D0
:100E700081608C93A5E3B0E0E5E3F0E080818B7FB7
:100E80008C93A5E3B0E0E5E3F0E08081877F8C936D
:100E9000A5E3B0E0E5E3F0E080818F7E8C93A8E3EA
:100EA000B0E0E8E3F0E080818F7D8C9363C0A5E340
:100EB000B0E0E5E3F0E0808180628C93A8E3B0E0ED
:100EC000E8E3F0E0808180618C93A5E3B0E0E5E3A6
:100ED000F0E080818E7F8C93A5E3B0E0E5E3F0E065
:100EE000808184608C93A5E3B0E0E5E3F0E080814D
:100EF000877F8C93A5E3B0E0E5E3F0E0808180613B
:100F00008C93A8E3B0E0E8E3F0E080818F7D8C93E0
:100F100031C0A5E3B0E0E5E3F0E0808180628C932E
:100F2000A8E3B0E0E8E3F0E080818F7E8C93A5E356
:100F3000B0E0E5E3F0E080818E7F8C93A5E3B0E044
:100F4000E5E3F0E080818B7F8C93A5E3B0E0E5E3FF
:100F5000F0E08081877F8C93A5E3B0E0E5E3F0E0EB
:100F6000808180618C93A8E3B0E0E8E3F0E08081C9
:100F70008F7D8C938981282F30E03D832C838C8159
:100F80009D818330910561F02C813D8124303105B4
:100F900009F457C08C819D818130910539F159C088
:100FA000809189008823B9F080E090E0B1D08091F1
:100FB0007A00882341F4A5E3B0E0E5E3F0E0808126
:100FC0008D7F8C935DC0A5E3B0E0E5E3F0E0808128
:100FD00082608C9355C082E090E09AD0A5E3B0E0A7
:100FE000E5E3F0E080818D7F8C934AC080917400AE
:100FF000909175002AE030E0B90183D185309105E8
:1010000040F4A5E3B0E0E5E3F0E0808182608C93FA
:1010100037C080917A00813021F080917A00882356
:1010200041F4A5E3B0E0E5E3F0E080818D7F8C93AF
:1010300027C0A5E3B0E0E5E3F0E0808182608C9317
:101040001FC0A5E3B0E0E5E3F0E0808182608C930F
:1010500017C080917A00813021F080917A00882336
:1010600041F4A5E3B0E0E5E3F0E080818D7F8C936F
:1010700007C0A5E3B0E0E5E3F0E0808182608C93F7
:1010800080917A00282F30E03B832A838A819B81DC
:1010900081309105E9F02A813B81223031052CF421
:1010A0008A819B81009761F02AC02A813B8122308E
:1010B0003105B1F08A819B8183309105C9F01FC051
:1010C000A8E3B0E0E8E3F0E080818E7F8C9317C066
:1010D000A8E3B0E0E8E3F0E080818B7F8C930FC061
:1010E000A8E3B0E0E8E3F0E080818D7F8C9307C057
:1010F000A8E3B0E0E8E3F0E08081877F8C93279657
:101100000FB6F894DEBF0FBECDBFCF91DF9108952B
:10111000DF93CF9300D00F92CDB7DEB7898389815B
:10112000282F30E03B832A838A819B81813091057F
:10113000C1F02A813B812230310511F18A819B81E6
:10114000009761F5A2E3B0E0E2E3F0E080818F7DFB
:101150008C93A2E3B0E0E2E3F0E080818F7B8C939C
:101160001DC0A2E3B0E0E2E3F0E0808180628C93F6
:10117000A2E3B0E0E2E3F0E080818F7B8C930EC0CD
:10118000A2E3B0E0E2E3F0E080818F7D8C93A2E304
:10119000B0E0E2E3F0E0808180648C930F900F90E8
:1011A0000F90CF91DF910895DF93CF9300D0CDB70B
:1011B000DEB79A83898389819A8128E532E0B90173
:1011C000A0D0CB0180938B0080918B008823D1F03D
:1011D00089819A812AE030E0B90193D0CB01482F70
:1011E00080918B00282F30E084EC9FEFBC01269F7C
:1011F000C001279F900D369F900D1124840F80937E
:101200008A0009C089819A812AE030E0B90179D049
:10121000CB0180938A0080918A009AE0692F65D083
:10122000892F8093760080918A0094E6692F5DD0A3
:10123000892F9AE0692F59D08093770080918B0095
:101240009AE0692F52D0892F8093780080918B008B
:101250008A3020F48AE0809379000BC080918B0063
:1012600094E6692F42D0892F9AE0692F3ED080936F
:1012700079000F900F90CF91DF910895DF93CF9376
:10128000CDB7DEB780E090E050D09C018091870020
:10129000909188002817390741F0209187003091FC
:1012A000880080E090E0B90145D0CF91DF910895AA
:1012B000DF93CF93CDB7DEB780E090E036D0909348
:1012C00088008093870080918700909188002FEF9D
:1012D0008F3F920739F488ED9EE0909388008093C9
:1012E0008700CCDFCF91DF910895991B79E004C08E
:1012F000991F961708F0961B881F7A95C9F7809555
:101300000895AA1BBB1B51E107C0AA1FBB1FA6174C
:10131000B70710F0A61BB70B881F991F5A95A9F79E
:1013200080959095BC01CD010895A8E1B0E042E020
:1013300050E005C012D0272F11C0DC01CB01FC0109
:10134000E199FECF06C0FFBBEEBBE09A31960DB22D
:101350000D9241505040B8F70895262FE199FECFE5
:101360009FBB8EBB2DBB0FB6F894E29AE19A0FBEDD
:0813700001960895F894FFCFE7
:02137800B80BB0
:00000001FF
